:100000000C9456000C9473000C9473000C947300C1
:100010000C9473000C9473000C9473000C94730094
:100020000C9473000C9473000C9473000C94730084
:100030000C9473000C9473000C9473000C94730074
:100040000C9473000C9473000C9473000C94730064
:100050000C9473000C9473000C9473000C94730054
:100060000C9473000C9473000C9473000C94730044
:100070000C9473000C9473000C9473000C94730034
:100080000C9473000C9473000C9473000C94730024
:100090000C9473000C9473000C9473000C94730014
:1000A0000C9473000C9473000C94730011241FBE05
:1000B000CFEFDAE0DEBFCDBF11E0A0E0B1E0E6E1D6
:1000C000FCE002C005900D92AE34B107D9F721E0F3
:1000D000AEE4B1E001C01D92A335B207E1F70E9482
:1000E000C5020C9409060C94000086E084B980E5F2
:1000F0008CBD08952D988FEF8EBD0DB407FEFDCFFA
:100100002D9A8EB50895982F86EF890F823010F0C2
:10011000903111F485E001C081E02D989EBD0DB4B1
:1001200007FEFDCF262FFB011EBC0DB407FEFDCF41
:100130009EB591939E2F921B9817B0F32D9A089518
:100140009F92AF92BF92CF92DF92EF92FF920F9366
:100150001F93CF93DF93CDB7DEB7C555D1090FB647
:10016000F894DEBF0FBECDBF1A821982FE0133960E
:1001700090E3DF011D929A95E9F77E01B1E5EB0E60
:10018000F11CB7010E948300982E1BAA67018E0103
:100190000D5C1F4F84E2A82E81E0B82E8C2D8E19A5
:1001A000891598F4F60181916F011F928F931F9327
:1001B0000F93BF92AF921F930F930E941F030FB62E
:1001C000F894DEBF0FBECDBFE9CF1F930F9382E13E
:1001D00091E09F938F938E010F5F1F4F1F930F939B
:1001E0000E941F03C8010E94AB020F900F900F9056
:1001F0000F900F900F90CB5ADF4F0FB6F894DEBFE1
:100200000FBECDBFDF91CF911F910F91FF90EF9067
:10021000DF90CF90BF90AF909F9008952D9880620F
:100220008EBD0DB407FEFDCF6EBD0DB407FEFDCF34
:100230002D9A0895249A259A2D9A2C988FEE95E55B
:100240000197F1F700C000006AE080E00E940E0113
:100250008FE99FE00197F1F700C0000008952D9805
:1002600080E58EBD0DB407FEFDCF83E78EBD0DB4D6
:1002700007FEFDCF2D9A08952D9890EA9EBD0DB4EE
:1002800007FEFDCF262FFB019E2F921B981730F4FF
:1002900091919EBD0DB407FEFDCFF6CF2D9A089526
:1002A0004F925F926F927F928F929F92AF92BF9286
:1002B000CF92DF92EF92FF920F931F93CF93DF9332
:1002C000CDB7DEB7EB970FB6F894DEBF0FBECDBF4C
:1002D0008091000190910101A0910201B091030170
:1002E00088AF99AFAAAFBBAF1A821982FE013396CD
:1002F00080E3DF011D928A95E9F7BE01685C7F4FBC
:1003000084E00E943C012C9AB8E2BA95F1F72C984F
:10031000412C512C32018CE2882E81E0982E02E192
:1003200011E0CE0101967C0197E3C92E91E0D92E10
:100330002EE3A22E21E0B22EAFECB7E01197F1F739
:1003400000C00000BE016D5C7F4F87E00E9483000B
:10035000823088F09F928F921F930F93FF92EF92BB
:100360000E941F03C7010E94AB020F900F900F90D5
:100370000F900F900F908BA985FF13C0DF92CF9243
:100380001F930F93FF92EF920E941F03C7010E94D9
:10039000AB020F900F900F900F900F900F9081E095
:1003A00001C080E09BA994FF12C0BF92AF921F933F
:1003B0000F93FF92EF920E941F03C7010E94AB02AE
:1003C0000F900F900F900F900F900F9081E0BFEF64
:1003D0004B1A5B0A6B0A7B0A811108C08FEF481623
:1003E00051046104710409F0A7CF06C09FEF4916BC
:1003F000510461047104C1F486E491E09F938F93EA
:1004000082E191E09F938F938E010F5F1F4F1F93A7
:100410000F930E941F03C8010E94AB020F900F9020
:100420000F900F900F900F90BE016D5C7F4F87E093
:100430000E9483006BA96F7087E00E940E01EB960B
:100440000FB6F894DEBF0FBECDBFDF91CF911F91E5
:100450000F91FF90EF90DF90CF90BF90AF909F9063
:100460008F907F906F905F904F900895CF93DF9320
:1004700000D000D0CDB7DEB769837A838B839C83AD
:100480002D9880E38EBD0DB407FEFDCFFE013196A1
:10049000CE01059621912EBD0DB407FEFDCFE817C4
:1004A000F907C1F71EBC0DB407FEFDCF2D9A0F90C2
:1004B0000F900F900F90DF91CF910895CF93DF931E
:1004C00000D000D0CDB7DEB769837A838B839C835D
:1004D0002D988AE28EBD0DB407FEFDCFFE01319648
:1004E000CE01059621912EBD0DB407FEFDCFE81774
:1004F000F907C1F71EBC0DB407FEFDCF2D9A0F9072
:100500000F900F900F90DF91CF91089562E385E0F7
:100510000E940E010E942F0164E08DE10E940E01F5
:100520006FE38CE10E940E0166E574E382E190E0E6
:100530000E94360266E574E382E190E00C945E026C
:100540009093CD008093CC0088E18093C9008EE029
:100550008093CA00089540E0242F30E0FC01019010
:100560000020E9F73197E81BF90B2E173F0760F4DD
:100570005091C80055FFFCCFFC01E20FF31F208112
:100580002093CE004F5FE8CF0895CF93DF93CDB790
:10059000DEB7E2970FB6F894DEBF0FBECDBF1A826A
:1005A0001982FE01339680E3DF011D928A95E9F7F7
:1005B00083E390E00E94A00284E091E09F938F93F8
:1005C00082E191E09F938F938E010F5F1F4F1F93E6
:1005D0000F930E941F03C8010E94AB020E94750086
:1005E0000E941A010E9486020F900F900F900F90A8
:1005F0000F900F9087E1C82E81E0D82E92E1E92E6E
:1006000091E0F92E0E945001DF92CF92FF92EF927B
:100610001F930F930E941F03C8010E94AB02BFEFFC
:1006200029E688E1B15020408040E1F700C0000099
:100630000F900F900F900F900F900F90E3CFAEE0C0
:10064000B0E0E5E2F3E00C94E0050D891E8986E058
:100650008C831A8309838FEF9FE79E838D83AE017E
:10066000475E5F4F6F89788DCE0101960E944103EE
:10067000EF81F885E00FF11F10822E96E4E00C94D4
:10068000FC05ABE0B0E0E7E4F3E00C94D2056C01CC
:100690007B018A01FC0117821682838181FFCCC114
:1006A000CE0101963C01F6019381F70193FD8591FE
:1006B00093FF81917F01882309F4BAC1853239F40F
:1006C00093FD859193FF81917F01853229F4B601D5
:1006D00090E00E943805E7CF912C212C312CFFE1CE
:1006E000F315D8F08B3279F038F4803279F0833218
:1006F000A1F4232D20611DC08D3261F0803369F497
:10070000232D216016C0832D8260382EE32DE460F6
:100710003E2E2AC0F32DF8601DC037FC2DC020ED01
:10072000280F2A3040F08E32B9F436FC81C1232DD7
:100730002064322E19C036FE06C08AE0989E200D35
:100740001124922E11C0EAE02E9E200D1124222E9B
:10075000F32DF0623F2E08C08C3621F4832D806883
:10076000382E02C0883641F4F70193FD859193FF3E
:1007700081917F018111B3CF982F9F7D9554933044
:1007800028F40C5F1F4F9FE399830DC0833631F02F
:10079000833771F0833509F059C021C0F801808199
:1007A00089830E5F1F4F88248394912C530113C0BB
:1007B0002801F2E04F0E511CF801A080B18036FEF6
:1007C00003C0692D70E002C06FEF7FEFC5010E948A
:1007D0002D054C018201F32DFF773F2E16C0280115
:1007E00022E0420E511CF801A080B18036FE03C009
:1007F000692D70E002C06FEF7FEFC5010E942205F6
:100800004C01F32DF0683F2E820133FC1BC0822D7A
:1008100090E088169906B0F4B60180E290E00E945C
:1008200038052A94F4CFF50137FC859137FE819184
:100830005F01B60190E00E94380521102A9421E062
:10084000821A91088114910471F7E8C0843611F07E
:10085000893641F5F80137FE07C0608171818281D8
:1008600093810C5F1F4F08C060817181072E000CBF
:10087000880B990B0E5F1F4FF32DFF763F2E97FFCE
:1008800009C090958095709561957F4F8F4F9F4FD0
:10089000F0683F2E2AE030E0A3010E947405882E04
:1008A000861845C0853731F4232D2F7EB22E2AE0DD
:1008B00030E025C0932D997FB92E8F36C1F018F402
:1008C000883579F0B5C0803719F0883721F0B0C08D
:1008D000E92FE061BE2EB4FE0DC0FB2DF460BF2EEB
:1008E00009C034FE0AC0292F2660B22E06C028E0B7
:1008F00030E005C020E130E002C020E132E0F80144
:10090000B7FE07C060817181828193810C5F1F4FA8
:1009100006C06081718180E090E00E5F1F4FA301EF
:100920000E947405882E8618FB2DFF773F2E36FE19
:100930000DC0232D2E7FA22E891458F434FE0BC037
:1009400032FC09C0832D8E7EA82E05C0B82CA32CA6
:1009500003C0B82C01C0B92CA4FE0FC0FE01E80DE5
:10096000F11D8081803321F49A2D997EA92E09C032
:10097000A2FE06C0B394B39404C08A2D867809F011
:10098000B394A3FC11C0A0FE06C0B21488F4280CD6
:10099000922C9B180EC0B21460F4B60180E290E075
:1009A0000E943805B394F7CFB21418F42B1802C084
:1009B000982C212CA4FE10C0B60180E390E00E9488
:1009C0003805A2FE17C0A1FC03C088E790E002C072
:1009D00088E590E0B6010CC08A2D867859F0A1FE1A
:1009E00002C08BE201C080E2A7FC8DE2B60190E07C
:1009F0000E943805891438F4B60180E390E00E9423
:100A000038059A94F7CF8A94F301E80DF11D80819F
:100A1000B60190E00E9438058110F5CF222009F43C
:100A200042CEB60180E290E00E9438052A94F6CFCB
:100A3000F6018681978102C08FEF9FEF2B96E2E14E
:100A40000C94EE05FC010590615070400110D8F740
:100A5000809590958E0F9F1F0895FC016150704006
:100A600001900110D8F7809590958E0F9F1F0895E3
:100A70000F931F93CF93DF93FB01238121FD03C0CD
:100A80008FEF9FEF2CC022FF16C046815781248133
:100A900035814217530744F4A081B1819D012F5F36
:100AA0003F4F318320838C93268137812F5F3F4FC7
:100AB0003783268314C08B01EC01FB010084F18590
:100AC000E02D0995892BE1F6D80116968D919C9120
:100AD0001797019617969C938E931697CE01DF91E8
:100AE000CF911F910F910895FA01AA27283051F153
:100AF000203181F1E8946F936E7F6E5F7F4F8F4F4F
:100B00009F4FAF4FB1E03ED0B4E03CD0670F781FAD
:100B1000891F9A1FA11D680F791F8A1F911DA11D92
:100B20006A0F711D811D911DA11D20D009F46894CB
:100B30003F912AE0269F11243019305D3193DEF673
:100B4000CF010895462F4770405D4193B3E00FD029
:100B5000C9F7F6CF462F4F70405D4A3318F0495D14
:100B600031FD4052419302D0A9F7EACFB4E0A695F7
:100B70009795879577956795BA95C9F70097610519
:100B8000710508959B01AC010A2E0694579547956F
:100B900037952795BA95C9F7620F731F841F951F64
:100BA000A01D08952F923F924F925F926F927F9275
:100BB0008F929F92AF92BF92CF92DF92EF92FF926D
:100BC0000F931F93CF93DF93CDB7DEB7CA1BDB0B19
:100BD0000FB6F894DEBF0FBECDBF09942A883988BE
:100BE00048885F846E847D848C849B84AA84B984C5
:100BF000C884DF80EE80FD800C811B81AA81B981D1
:100C0000CE0FD11D0FB6F894DEBF0FBECDBFED01E4
:060C10000895F894FFCFE7
:100C1600DEADBEEF50726F6772616D2073746172E4
:100C2600740025730D0A0074657374206D65737303
:100C360061676500257330782578200072656164E8
:100C4600206572726F720054582066696E006D617D
:0E0C560078207265740074696D656F757400A6
:00000001FF
